:020000040000FA
:04000000803186289D
:0800080020008331282B820740
:100010000034013402340334043405340634073424
:10002000083409340A340B340C340D340E340F34D4
:100030000A340B340C340D340E340F348207303450
:10004000313432343334343435343634373438346C
:1000500039344134423443344434453446346134D1
:10006000623463346434653466342030B200031083
:10007000A80DA90DAA0DAB0D0310A00DA10DA20D89
:10008000A30D031C4B282408A8072508A93D260812
:10009000AA3D2708AB3DB20B372808002030B2003C
:1000A000A401A501A601A7010310AC0DAD0DAE0D75
:1000B000AF0D0310A00DA10DA20DA30DA40DA50D54
:1000C000A60DA70D27082B02031D702826082A025B
:1000D000031D702825082902031D70282408280202
:1000E00003197428031883282808A4022908031C6C
:1000F000290FA5022A08031C2A0FA6022B08031C9D
:100100002B0FA7022C14B20B5428080021008C10CE
:100110000C128C12E9282500BD0023009E019E16BA
:100120001E151E129F119D011D169D1725003D08CD
:1001300023009B009C0108002500BC0023009E18A2
:10014000A2289E2825003C0823009A0008002300CE
:100150001D1DAE289D139D1725003B1023009D1CDF
:10016000B6281D121D1625003B10BE282000911A2E
:10017000BC2825003B10BE2825003B143B18C32893
:100180002000201008002000201408002300190877
:1001900008002500BA0023009100951315131514CB
:1001A000130808002500B800230091002500390835
:1001B000230093009513151315158B1355309600D6
:1001C000AA30960095148B171511951CE828E52880
:1001D00008000E108E100E118E118331312B22006B
:1001E0008E118E109D0124009512F03015050138F6
:1001F000950015121417FF302000BC009111220049
:100200008E15240095162100911508002000911DDF
:10021000502922008C1620003C08031D14292400BC
:1002200091012000BC0A4C293C03031D1D29FF300D
:10023000240091002000BC0A4C2902303C02031D1E
:100240002A2922008E142000BC0A22008E102400CD
:1002500091014C2903303C02031D34293E0824003F
:1002600091002000BC0A4C2904303C02031D3F29A8
:10027000FF303D06240091002000BC0A4C290530C7
:100280003C02031D4B2922008E14FF302000BC00CD
:1002900022008E104C293C0A2000911122008C1261
:1002A000090020001C1187309C05FC301C05033818
:1002B0009C000E309B009A01BF01F03025001A050A
:1002C0000A389A00210091140B178B1720001C1577
:1002D0000800911C062922000C162000B7010F30DF
:1002E0003F020319772903187729B801AF291E3077
:1002F0003F0203198029031880290130B800AF2973
:100300002D303F0203198929031889290230B800CA
:10031000AF293C303F020319922903189229033078
:10032000B800AF294B303F0203199B2903189B29C2
:100330000430B800AF295A303F020319A42903182A
:10034000A4290530B800AF2969303F020319AD294F
:100350000318AD290630B800AF290730B8003808B7
:10036000031DD6293F0AB600B90107303902031927
:10037000BB290318CB290310B70CA03084008501DA
:1003800039088407000836020319C8290318C92947
:10039000B717B90AB5293708BA00BB013A08BD003A
:1003A00001303B04BE00BF0A8331042B3803823185
:1003B000031D012A0E303F02B6000830B9000F308D
:1003C000390281310319E6290318F6290310B70C05
:1003D000A03084008501390884070008360203191B
:1003E000F3290318F429B717B90ADF293708BA0027
:1003F000BB013A08BD0002303B04BE00BF0A833196
:10040000042B02303802031D2B2A1D303F02B60098
:100410001030B900173039020319102A0318202AA6
:100420000310B70CA0308400850139088407000848
:10043000360203191D2A03181E2AB717B90A0A2AF9
:100440003708BA00BB013A08BD0004303B04BE00C7
:10045000BF0A8331042B03303802031D552A2C3088
:100460003F02B6001830B9001F30390203193A2A8A
:1004700003184A2A0310B70CA030840085013908FC
:100480008407000836020319472A0318482AB717B9
:10049000B90A342A3708BA00BB013A08BD0008304F
:1004A0003B04BE00BF0A8331042B04303802031D15
:1004B0007F2A3B303F02B6002030B9002730390296
:1004C0000319642A0318742A0310B70CA03084009F
:1004D000850139088407000836020319712A0318B8
:1004E000722AB717B90A5E2A3708BA00BB013A0860
:1004F000BD0010303B04BE00BF0A8331042B053021
:100500003802031DA92A4A303F02B6002830B9003C
:100510002F30390203198E2A03189E2A0310B70CB4
:10052000A0308400850139088407000836020319C9
:100530009B2A03189C2AB717B90A882A3708BA00D9
:10054000BB013A08BD0020303B04BE00BF0A833126
:10055000042B06303802031DD32A59303F02B6005F
:100560003030B900373039020319B82A0318C82AC5
:100570000310B70CA03084008501390884070008F7
:1005800036020319C52A0318C62AB717B90AB22AB0
:100590003708BA00BB013A08BD0040303B04BE003A
:1005A000BF0A8331042B073038028331031D042B2B
:1005B00068303F02B6003830B9003F30390282312E
:1005C0000319E42A0318F42A0310B70CA03084009E
:1005D000850139088407000836020319F12A031837
:1005E000F22AB717B90ADD2A3708BA00BB013A0860
:1005F000BD0080303B04BE0077303F028331031DD5
:10060000032BBF01042BBF0ABC01911591102200DE
:100610000C12813106292800171187301705783808
:100620009700FC301705033897004D309600950170
:10063000F03026001A050A389A0020009310220094
:100640006110210093140B178B1728001715080051
:1006500081312000931C692922006114200093102D
:10066000692928238631EB2E36082000C00025009A
:1006700037082000C100080003102000410C2500AD
:10068000AB002000400C2500AA000310AB0CAA0C04
:100690002A08200040062500AC002B082000410657
:1006A0002500AD0003102000410C2500AF00200004
:1006B000400C2500AE000310AF0CAE0C0310AF0CC5
:1006C000AE0C2E082C06B0002F082D06B10003102A
:1006D0002000410C2500B3002000400C2500B20092
:1006E00004302000A00003102500B30CB20C200041
:1006F000A00B732B250032083006B40033083106F6
:10070000B50001303405A800A90103102000410CF8
:100710002500AB002000400C2500AA00AC01AD0173
:100720002818AD172C082A042000C00025002D0829
:100730002B042000C10008003C23E13020004002CF
:10074000A000AC30410220048331031DAA2BA0017C
:10075000A10108004008A0004108A10008002000F5
:10076000C20108002400ED00EF012500271016301B
:1007700024006F022500A7100319C02B031CA71427
:1007800027182711271C2715A715A718271DA711FC
:10079000A71DE42B24006F0880311E202000A0003C
:1007A00024006D08200020028331031DE12B24006A
:1007B0006F08803107202400EE00250027148331C4
:1007C000B72B2400EF0AB72B2718E92B20002010A5
:1007D000EB2B2000201424006E0808002400EA00FF
:1007E000EB016C100F30EA0584316C180B2C6B0890
:1007F000803107202000A00024006A082000200289
:100800008431031D072C24006C148331F42B240045
:10081000EB0A8331F42B6B0880311E282500201051
:1008200020004208031D382C8031A720843120008D
:1008300020181D2C250020111F2C25002015863185
:10084000201DE12E2000C6010530C3008031C620E6
:100850002000C400213044028431031D332C0130B8
:10086000C2008631E12E4E3080319C208631E12E4F
:100870004203031D612C8031A72084312000201801
:10088000442C2500A012462C2500A0168631A01E5F
:10089000E12E8031C6202000C40030304402C30065
:1008A00005304302843103195B2C03185B2C0430A0
:1008B000C2008631E12EC2014E3080319C2086314B
:1008C000E12E02304202031D912C8031A720843199
:1008D000200020186E2C25002110702C25002114DA
:1008E0008631211CE12E8031C6202000C4008331D6
:1008F000B2232000CB0084312018812C2500A110C8
:10090000832C2500A114A11C8A2C03302000C200D6
:100910008631E12E2000C2014E3080319C2086318C
:10092000E12E03304202031DE22C8031A7208431E6
:10093000200020189E2C2500A111A02C2500A11517
:100940008631A11DE12E8031C6202000C400413037
:10095000460284310319DC2C0318DC2C4408833153
:10096000B2232000CC0084312018B92C2500A1121C
:10097000BB2C2500A116A11ED52C20004B0EF03952
:100980002400E80020004C08240068042000C50072
:100990002030840001308500460884074508800027
:1009A000C60A0430C2008631E12E2000C2014E305A
:1009B00080319C208631E12EC2014E3080319C2056
:1009C0008631E12E043042028631031DE12E803152
:1009D000A720843120002018F02C2500A113F22C30
:1009E0002500A1178631A11FE12E8031C6202000ED
:1009F000C4000D30440225002210031922140A30CD
:100A0000200044022500A2100319A2142211221C66
:100A1000A218221586312219E12E2C302000440222
:100A20008531031D172D0230C2008631E12E23309F
:100A300044028631031DDD2E43088531031D942DAC
:100A400020304602031D8F2D2200E1142000C90131
:100A500049084602250023100319302D03182314DA
:100A6000A310231C382D2200E11C382D2500A314CF
:100A70002500A31C662D2030840001308500200055
:100A8000490884070008C500450E0F392400E80016
:100A90000F30680225002311031D031C23150F309E
:100AA000200045052400E9000F3069022500A3114C
:100AB000031D031CA3152200E11025002319A31D0B
:100AC000632D2200E1142000C90A282D2200E11C18
:100AD0008A2D2000C9014908460285310319832D5A
:100AE000031C832D203084000130850049088407D1
:100AF00000082500B900200049088031D2202000DC
:100B0000C90A85316B2D593080319C202500201475
:100B10008631D92E4E3080319C208631D92E4E30F0
:100B200080319C208631D92E43038631031D242E2B
:100B30004030220020022500A313031D031CA3172D
:100B4000200046032400E800220020082400680258
:100B50002500241003192414A414A31B241CA4107E
:100B6000A41C1F2E2200E11401302000C9004908F6
:100B700046022500241185310319C02D03182415C0
:100B8000A411241DC82D2200E11CC82D2500A41588
:100B90002500A41DF22D20308400013085002000A6
:100BA000490884070130000225002412031D0318A0
:100BB0002416203084000130850020004908840775
:100BC000403000022500A412031D031CA4162200BD
:100BD000E1102500241AA41EEF2D2200E1142000AC
:100BE000C90AB72D86312200E11C1A2E2F302000B1
:100BF000C800C9014908460286310319132E031C97
:100C0000132E203084000130850049088407000835
:100C10002500B900200048088031D2202000C90AF0
:100C2000C80A8531FA2D593080319C2025002014C6
:100C30008631D92E4E3080319C208631D92E4E30CF
:100C400080319C208631D92E02304302031D532E61
:100C50000D304602031D4E2E2030C800C901490840
:100C600046020319472E031C472E20308400013012
:100C700085004908840700082500B90020004808BD
:100C80008031D2202000C90AC80A86312F2E59305F
:100C900080319C20250020148631D92E4E308031A1
:100CA0009C208631D92E03304302031D712E7F30E4
:100CB000220020052000C5004603031D6C2E4508B8
:100CC0002500B90070308031D220593080319C200D
:100CD000250020148631D92E4E3080319C2086315B
:100CE000D92E04304302031DD22E4608031DCD2EFB
:100CF000593080319C202000C7010F304705240067
:100D0000E80068088631031DA42E0D3080319C2038
:100D10000A3080319C202000470E0F392400E80063
:100D20008331EE232400E90080319C202000470815
:100D30008331EE232400E80080319C203A3080315A
:100D40009C20203080319C20200047088031C92021
:100D50002000CA004A0E0F392400E8008331EE2338
:100D60002400E90080319C2020004A088331EE23D2
:100D70002400E80080319C20203080319C2020001D
:100D8000C70A47088631031D7D2E0D3080319C2017
:100D90000A3080319C208631D92E4E3080319C2003
:100DA0008631D92E05304302031DD92E4E308031B5
:100DB0009C202000C2018631E12EC2014E308031DC
:100DC0009C20863125002018E82E200020100800E5
:100DD0002000201408002100991787301905703869
:100DE0009900FC3099053F3024008C003F308E0084
:100DF0002100951323008C018E0121009D019E018D
:100E0000220091019201930194018931DE29210090
:100E1000EE00EF01A030840085016F0884076E08A2
:100E20008000EF0A40306F02031D0A2F08002100E6
:100E3000ED0183319C23200020082400E0002000E5
:100E400021082400E1002000590A2400E200E30107
:100E500062082000A800240063082000A900AA015D
:100E6000AB01240060082000A000240061082000DD
:100E7000A100A201A30180314E20200024082400FB
:100E8000E400200025082400E50020005A08240082
:100E9000E600E701640866072000CF00240065082B
:100EA000673D2000D000A0308400850121006D083E
:100EB000840720004F0880002100ED0A40306D02B9
:100EC0008731031D192F080020308031C9202000F0
:100ED000D100FA30510287310319772F031C772F85
:100EE0007030EC001730ED00EE01EF019D2F51083E
:100EF0002200E800E901EA01EB0168082000A000F7
:100F0000220069082000A10022006A082000A20037
:100F100022006B082000A3007030A4001730A50049
:100F2000A601A7018031352020002808EC002908FF
:100F3000ED002A08EE002B08EF0021308031C92097
:100F40002000D100FA30510287310319AF2F031C62
:100F5000AF2FB8302100E0000B30E100CC2F51085A
:100F60002200E800E90168082000A00022006908CA
:100F70002000A100A201A301DC30A4000530A500DF
:100F8000A601A70180313520200028082100E000BB
:100F9000200029082100E10022308031C9202000F2
:100FA000D100FA30510287310319DF2F031CDF2FE4
:100FB000E0302100E2002E30E3008831042851089F
:100FC0002200E800E90101306807EA000030031858
:100FD00001306907EB006A082000A00022006B08BE
:100FE0002000A100A201A301DC30A4000530A5006F
:100FF000A601A70180313520200028082100E20049
:10100000200029082100E30023308031C92020007E
:10101000D100FA305102883103191428031C142816
:101020000A302100E500172851082100E50024308E
:101030008031C9202000D1000F30510288310319BE
:101040002728031C27280F302100E9002A285108EF
:101050002100E9002200E111611225308031C92010
:101060002000D100FA305102883103193C28031CBA
:101070003C283230D7003E285108D7005708D60008
:1010800026308031C9202000D1000F305102883134
:1010900003194F28031C4F280130DA00512851084A
:1010A000DA0027308031C9202000D1000F305102F2
:1010B000883103196028031C60280330D900622896
:1010C0005108D90028308031C9202000D1000F30CC
:1010D0005102883103197128031C71280130D8008E
:1010E00073285108D80029308031C9202000D10050
:1010F000FA305102883103198628031C86285030A3
:10110000DF004630E000E101E201AC285108220096
:10111000E800E901EA01EB0168082000A0002200D4
:1011200069082000A10022006A082000A200220015
:101130006B082000A3007030A4001730A500A601A2
:10114000A7018031352020002808DF002908E000B1
:101150002A08E1002B08E2002A308031C920200053
:10116000D100FA30510288310319BE28031CBE2871
:101170006430DB00DC01DD01DE01C3285108DB0047
:10118000DC01DD01DE012B308031C9202000D100DF
:10119000FA30510288310319D428031CD428E830CE
:1011A000E5000330E600ED2851082200E800E901DF
:1011B00068082000A000220069082000A100A20108
:1011C000A3016430A400A501A601A7018031352048
:1011D00020002808E5002908E6002C308031C920CD
:1011E0002000D100FA30510288310319FE28031C77
:1011F000FE286430E700E801893101295108E70041
:10120000E80170308031C9202000D1002200ED16A5
:10121000031DED122000510A22006D1303196D17F2
:10122000ED13ED1E6D1BED178931ED1F1F296211A6
:10123000E112E11761136210E210E2115729013047
:10124000200051052200E800E1160319E1120430E4
:10125000200051052200E800E1170319E1130230D4
:10126000200051052200E8006117031961130830BE
:10127000200051052200E8006214031962101030AA
:10128000200051052200E800E2140319E21020308A
:10129000200051052200E800621503196211403058
:1012A000200051052200E800E2150319E211621D39
:1012B0006729E112E1136113E210E2110030873176
:1012C00007272000E901E301E4018931C729E11E74
:1012D0009F292000D301D201403053020319C729AE
:1012E0000318C72952088031C9202200E800680E7F
:1012F0000F39E900A03084008501200053088407DD
:101300000F302200690580002000530A2200E80007
:10131000200052088031C9202200E9000F30690501
:10132000EA00A03084008501680884070F306A0550
:10133000800002302000D307D20A89316C29621C58
:10134000A529873117278931C7292000D3010A3001
:10135000A800A901AA01AB015308A000A101A201A4
:10136000A30180314E20200024082200E800A03094
:10137000840085012000530884072200680A800049
:101380002000D30A403053028931031DA7292000D1
:10139000D301A03084008501530884070008A00011
:1013A0002030840002308500530884072008800024
:1013B000D30A40305302031DC92908008E11FE30A4
:1013C0008031C9202000CD00FF308031C9202000AD
:1013D000CE004D084E0422006216031D621220004A
:1013E0004D0AA0004E0A20042200E2120319E21660
:1013F0006213621EE21A62178A31621F042AE13008
:101400002000CD00AC30CE0020004D082500B600F5
:1014100020004E082500B7008331342383319C23FC
:1014200020002008CD002108CE004D082500B9007D
:10143000FE308031D22020004E082500B900FF3058
:101440008031D2208331AF238731642767308031E8
:101450008B208031EF208131512183310B2380316A
:10146000A7208A3120002018382A2200E2133A2AC5
:101470002200E217E21F4B2A84310E248A31200019
:101480002018452A22006310472A22006314631C97
:101490004B2A873164278A312200611C2F2A611070
:1014A0008C14621DAD2A200063086404031DA92A60
:1014B0006508E3006608E4002200621C632A8731A5
:1014C00017278A31AD2A20006908031D702A0F30C2
:1014D000EA008731072701302000E9008A31AD2A70
:1014E0006903031D802AEA036A0887310727200061
:1014F0006A088A31031DA82A0230E900EB01AD2AEF
:1015000002306902031DAD2A6708E3006808E400A1
:10151000A030840085016B0884070008031D982A09
:10152000A030840085016B0884070F308000A82A52
:10153000A030840085016B088407800140306B0275
:101540000319A62A0318A62AEB0AA72AE901AD2A3D
:10155000AD2AE303630A0319E4032200611A64104D
:10156000611E6414E414E11B641CE4108B31E41C60
:10157000362B20005608031D352B5708D600833123
:101580009C2320002008CD002108CE003F304D05CF
:10159000D400A03084008501540884070008D500D9
:1015A0002200E415031DE4116416E218E41D641220
:1015B0008B31641A362B7F3020004E028A31031D96
:1015C000E32AFF304D028B310319012B031C012B41
:1015D000550858072300E000200059028A310319FA
:1015E000F82A031CF82A5508580780008B31362B3F
:1015F000A0308400850154088407590880008B318D
:10160000362B2200E21D152B20308400023085008D
:101610002000540884070008A000A0308400850141
:101620005408840720088000362B20005A085807E9
:101630002300E000200055082300600203192C2B32
:1016400003182C2BA0308400850120005408840747
:10165000580855028000342BA030840085012000FA
:10166000540884075A088000362BD6032200611ADA
:10167000E510611EE5146515E218E51C6511651D90
:10168000952B20005F08600461046204031D8D2B0C
:1016900083319C23200020082300E0002000210843
:1016A0002300E1003F3060052000D400A03084001A
:1016B0008501540884070008D50055088B310319AB
:1016C000952B5B08DF005C08E0005D08E1005E0828
:1016D000E200A0308400850154088407550380008F
:1016E000220061152000D301A03084008501530839
:1016F0008407000803197E2B220061112000D30A01
:1017000040305302031D742B2200611D952B611381
:10171000E210E1136211E211952B0130DF02031C8C
:10172000E002031CE102031CE2028C312200611F73
:10173000DC2C611A942C20006C086D046E046F047C
:10174000031D8B2C2200621C3C2C2100600823000E
:10175000E000210061082300E100E201E3018331A0
:101760009C23200020082300E400200021082300FF
:10177000E500E601E701210062082300E8002100FE
:1017800063082300E900EA01EB0168082000A800D3
:10179000230069082000A90023006A082000AA008D
:1017A00023006B082000AB00230064082000A00089
:1017B000230065082000A100230066082000A20085
:1017C000230067082000A30080314E202000240859
:1017D0002300EC00200025082300ED00200026084F
:1017E0002300EE00200027082300EF0060086C07AC
:1017F0002000EC00230061086D3D2000ED00230077
:1018000062086E3D2000EE00230063086F3D20005B
:10181000EF0083319C23200020082300E0002000FB
:1018200021082300E1003F306005E200620A210048
:10183000E600EB002000D3018C31352C83319C2352
:10184000200020082300E000200021082300E10000
:10185000A0308400013085002000530884073F3009
:101860002300600580002000D30A530821006B028A
:101870008C31031D1E2C822C210060082000EC00FE
:10188000210061082000ED00EE01EF012F308031D2
:10189000C9202100E60022006615031966114030B8
:1018A000210066022200E611031D031CE6156616E0
:1018B0006619E61D66128C31661E802C21006608B2
:1018C000EC002000D301792C303020005307230096
:1018D000E0008031C9202300E100A0308400013005
:1018E0008500200053088407230061038000200046
:1018F000D30A530821006C028C31031D642C822C06
:101900002100E60166080319DC2CE701E40122004E
:10191000E1116116DC2C0130EC02031CED02031C0A
:10192000EE02031CEF02DC2C21006408031DDB2CFB
:10193000670866020319D82C031CD82C2200E11971
:10194000C12CA03084000130850021006708840785
:1019500000082000D400A0308400850154088407CA
:1019600000082100E800A030840085012000540810
:1019700084072100690880006508E4002200E11561
:10198000DC2CA0308400013085002100670884072A
:1019900000082000D400A03084008501540884078A
:1019A0002100680880002200E1112100E70ADC2CF8
:1019B00022006112DC2CE40322008C108A312F2AD1
:020000040001F9
:02000E00843F2D
:02001000FF1FD0
:00000001FF
